:020000040000FA
:100000003028000000000000F200030E8301F5001C
:100010000A08F4008A010408F300831203138C1EFB
:1000200027281A08981C18281A08181218160D28BC
:1000300083160313F600A10AE3302102031D2228D0
:10004000A230A10021088400760880000D287308E2
:10005000840074088A00750E8300F20E720E090087
:100060008301831603132730810000308C00003099
:100070008D000B30850000308600B03087000430E2
:100080009F0083120313003085000030860000308B
:100090008700C0308B00003090008C0197019D01DB
:1000A000203084008001840A6D300402031C522831
:1000B000C6232824042183160313A230A100A00024
:1000C0008C168312031307142830A5005C30A60099
:1000D0008F30A7000230A800332157217421031C60
:1000E0006E28A800A81BBE287421031C7428A70032
:1000F0007421031C7828A6007421031C7C28A50009
:1001000057217421031C8128A0007039A100210C03
:100110003839860020080739820796289A289E28B1
:10012000A228A628AC28B228B8286E28C9302021D9
:100130001B216E28C13020211B216E28D1302021A7
:100140001B216E28D93020211B216E28C930202187
:100150001B2124081B216E28C13020211B212408CB
:100160001B216E28D13020211B2124081B216E2841
:10017000D93020211B2124081B216E2828080F3983
:100180008207D228D328D428D528DC28D628EA28E4
:10019000F0286E286E286E286E286E286E286E282D
:1001A0008E296E28A628AC28B228B82861302021D4
:1001B0001B2124081B216E287421031CDC28A700A6
:1001C0007421031CE028A6007421031CE428A50068
:1001D00073216E287421031CEA2886001B216E28D7
:1001E0007421031CF028A8007421031CF428A70024
:1001F0007421031CF828A6007421031CFC28A50008
:100200005721AA301B216E28831203130716831669
:10021000031307120A309900181598168312031356
:10022000181698170712080007128C1E15291A08AD
:100230000800871A19290C1E1B2999000800C130D3
:100240009F002E211F151F192329831603131E0833
:1002500083120313A4001E08A30008000730A000A7
:10026000A00B302908002830A5005C30A6008F3094
:10027000A7000230A8008714000000000000000062
:1002800000000000871000000000000000000000D7
:10029000871500000000871100000000071500000E
:1002A00000000711000000005721572108002530E9
:1002B00084000430AC000008AE006621840AAC0B58
:1002C0005B29AE0166210715071108000830AD0053
:1002D000AE0C031C6D2907146E29071087158711B2
:1002E000AD0B6829080008008316031321082002BB
:1002F00083120313031D7E290310080083160313C2
:10030000A00AE3302002031D8729A230A0002008A4
:1003100084000008831203130314080013227421BD
:10032000031C8F29E80060306802031813224F3045
:1003300084004E08840768088000CE0A4F08773A88
:10034000031DA9294E08163A031DA9292B140D23B4
:10035000112A4F08663A031DB3294E080A3A031DB5
:10036000B3297623112A4F08783A031DBE294E0877
:10037000163A031DBE292B100D23112A4F086D3A82
:10038000031DC8294E08013A031DC8296523112AF7
:100390004F08653A031DD2294E080D3A031DD22994
:1003A0008623112A4F08763A031DDC294E08013AAC
:1003B000031DDC29C223112A4F08723A031DE629C6
:1003C0004E08023A031DE629C723112A4F08613A55
:1003D000031DF1294E08193A031DF1292B100B2397
:1003E000112A4F08623A031DFC294E08193A031DD1
:1003F000FC292B140B23112A4F08733A031D062ADC
:100400004E08013A031D062AB223112A4F086F3AFB
:10041000031D102A4E08023A031D102AC523112A73
:100420008F2913226E289D220800D201D301D40106
:10043000D501D601D701CE01CF01D001D1010800ED
:100440001522480884000008CE00840A0008CF0066
:10045000840A0008D000840A0008D100840A000839
:10046000D2002830AC000310D20CD10CD00CCF0C31
:10047000CE0CD70CD60CD50CD40CD30C4E3084003B
:100480000530AD00801F462A30308002801D4A2A88
:1004900003308002840AAD0B422AAC0B332A480891
:1004A000840053088000840A54088000840A550898
:1004B0008000840A56088000840A570880000800DB
:1004C0002E08D8002F08D9003008DA003108DB00E8
:1004D0003208DC002030D6005830C8006030C90037
:1004E000CF010310D50CD40CD30CD20C031C912AD1
:1004F0000830D000480884000008CE004908840075
:100500004F08CF018007031C872A0130CF004E0817
:100510008007031C8D2A0130CF00C80AC90AD00BFE
:100520007A2A0310D80DD90DDA0DDB0DDC0DDD0DA7
:10053000DE0DDF0DD60B6C2A08004E3084008001E2
:10054000673004020319A62A840A9F2A080050086B
:100550000F39B800510EF039B70052080F39B704FF
:10056000530EF039B60054080F39B604550EF03961
:10057000B50056080F39B504570EF039B4005808C5
:100580000F39B4040800BD01590EF039BC005A08F7
:100590000F39BC045B0EF039BB005C080F39BB049B
:1005A0005D0EF039BA005E080F39BA045F0EF039FB
:1005B000B90060080F39B9040800C001C101C201C7
:1005C000610EF039BF0062080F39BF04630EF039C5
:1005D000BE0064080F39BE040800C401C501C6018D
:1005E000C70165080F39C404660EF039C3006708F7
:1005F0000F39C30408004308EB004408EC000F3037
:10060000EA00EA0B012BEB0BFF2AEC0803190A2B7B
:10061000EC03FF2A0800ED220F2BC301C40183164F
:10062000031384309F0083120313A722C322DD2209
:100630003430C80020223930C80020223E30C800A3
:1006400020224330C80020229D223508D3003408E0
:10065000D2003608D4003708D5006022DB23C30857
:10066000031D362BC408031D362B372BFB223908FC
:10067000B4073A0803183A0FB5073B0803183B0FB5
:10068000B6073C0803183C0FB7079D223508D30076
:100690003408D2003608D4003708D5006022E92398
:1006A00024081B2123081B21E72324081B212308DE
:1006B0001B21DB23BE033E0A0319BF03BE08031D33
:1006C0002F2BBF08031D2F2B080083160313843024
:1006D0009F0083120313EB2324081B2123081B21F3
:1006E000E72324081B2123081B210800A7223430FC
:1006F000C80020229D223508D3003408D2003608D5
:10070000D4003708D5006022DB2308005008D3232B
:10071000B200B20E5108D323B2045208D323B10061
:10072000B10E5308D323B1045408D323B000B00E44
:100730005508D323B0045608D323AF00AF0E570893
:10074000D323AF045808D323AE00AE0E5908D323E9
:10075000AE045A08D323B300B30E5B08D323B3040B
:100760003524302808301B2169081B218316031308
:1007700084309F0083120313E42324081B212308E1
:100780001B21080077301B210800080008005008D2
:10079000E90005128512051169180516E918851674
:1007A000691905150800CE0041304E02303003189B
:1007B00037304E0208006508A6006408A5006608E8
:1007C000A7006708A8005729A401A30108009930D1
:1007D000EE2B2B18ED2B8930EE2B81309F00FC2364
:1007E0001F151F19F12B831603131E088312031301
:1007F000A4001E08A3000800C830CE00CE0BFE2BBC
:100800000800831603178C18032C83120317700833
:100810008D0071088C00831603178C130C158B1335
:1008200055308D00AA308D008C148B170C1183125B
:10083000031308008312031770088D008316031733
:100840008C130C14831203170C0883120313080073
:100850000630AC002E3084000030F0001A248000F6
:10086000840AF00AAC0B2E2C08000630AC000030D5
:10087000F0002E3084000008F1000124840AF00A00
:10088000AC0B3B2C08001A30EC007730EB005530F5
:10089000EA00EA0B492CEB0B492CEC0B492C080025
:0208A000000056
:02400E00723FFF
:0C4200004D00D00017005C002200000000
:00000001FF
